:10000000B201D428A2008316071383120930A3007B
:1000100003101520A20CA30B09280314152000308F
:10002000A1006430B3200314CF2803181A2800005D
:1000300007131C2807171C280130A1009330B32890
:10004000A7008910091009108316891009100910DA
:100050000F30880583122708B2184C283A30A100C7
:100060009830B3203330A60060201330A1008830D0
:10007000B32060206430B22060206430B22022308F
:10008000A600602028304B200C304B2006304B203F
:10009000B21427084C283214A600321C5A28091022
:1000A000033C031C5F285F200730A100D030B32041
:1000B000031408003214FE3C0319CF280914321C23
:1000C000321089140F3088052608F0398804891009
:1000D000A60E321860283230B220031408006400E3
:1000E0007F2003186F288A200830A3008B207F20F0
:1000F000A20C7A28A30B76288B2022080800360849
:1001000084003408841780048413000533193406EE
:10011000FF3E08003317330D0639A0009920A100D7
:10012000A00A9920331FB3283313A0000230CA203D
:10013000B32800308A002008820701347534033464
:10014000153400343C340C34D934A301A200FF3000
:10015000A207031CA307031CCF280330A100DF3034
:10016000B320A728A101E83EA000A109FC30031C90
:10017000BC28A0070318B928A0076400A10FB9285C
:100180002018C228A01CC6280000C628080003109A
:10019000A10CA00CFF3E0318C7282008CF2883130A
:1001A0000313831264000800831607309F00831234
:1001B000091183160911643083128A01A520FE30CB
:1001C0008A01202001308A0120200530B60010303D
:1001D000B4000130B3008A016F20B800B9013808BB
:1001E0008A0102203808B8003908B90020308A0195
:0C01F000202038088A0120208A01E52820
:02400E00753DFE
:00000001FF
